:020000040800F2
:10500000201A0020D5500008518C0008198400088F
:105010000000000000000000000000000000000090
:10502000000000000000000000000000ED980008F3
:105030000000000000000000C9910008099A000863
:10504000E7500008E7500008E7500008E750000864
:10505000E7500008755B0008E7500008E7500008BB
:1050600000000000E7500008995A0008E7500008C7
:10507000E75000087188000800000000E7500008B1
:1050800000000000E75000080000000000000000E1
:10509000E750000800000000E7500008E750000853
:1050A000E7500008E7500008E7500008E5A30008B3
:1050B000E7500008E7500008000000000000000072
:1050C0000348854600F060FC0048004741B20008F4
:1050D000201A00200448804704480047FEE7FEE706
:1050E000FEE7FEE7FEE7FEE7A59A0008C1500008CC
:1050F00030B50B46014600202022012409E00D4670
:10510000D5409D4205D31D469540491B25469540F7
:1051100040191546521E002DF1DC30BDF0B51FB40C
:105120000646002082B005464024019100901BE015
:10513000019922460F46304600F04EFB049A059B2B
:10514000801A994110D310461946224600F034FBCC
:10515000361A8F410197224601200021009F00F05E
:105160002BFB38184D4100902046641E0028DFDCE0
:10517000019B00982946324607B0F0BD03460B4319
:105180009B0703D009E008C9121F08C0042AFAD2FD
:1051900003E00B780370401C491C521EF9D2704783
:1051A000D2B201E00270401C491EFBD270470022BF
:1051B000F6E710B513460A4604461946FFF7F0FF16
:1051C000204610BD30B504460020034600E05B1CBD
:1051D000934203D2E05CCD5C401BF8D030BDF8B503
:1051E00002464A40D40F42004B0052085B089A42E4
:1051F00002D20246084611464A0023D0C30D4A0097
:10520000DDB2120EAD1A202D35DA49020126490A07
:10521000F6058A19002C00D0524220214F1B11465E
:10522000B9402A411018C20D9A4221D0002C17D043
:10523000012D08DCDA05801AD20F8019D207DBB203
:1052400000F0F6FAF8BDDA05801A012340001B06CB
:10525000C01880185A428018CA0F1043490007E04E
:105260004908C2071143DA05801A801940088018DE
:1052700000F0D6FAF8BD61000122511A001BF7E7D1
:105280000122D2075140AAE70122D2075040A6E7E7
:1052900070B502464A40D50F40004A00ED0740086D
:1052A0005208002814D0002A12D0C40DD30D410298
:1052B0000120C0055202490A520AE41A09181218BC
:1052C0007D34914201D3641C00E04900002C01DAD6
:1052D000002070BD0023914201D3891A0343400886
:1052E00049000028F7D100290AD0914202D10121BA
:1052F000C90705E0914201D2012101E00121C94322
:10530000E005C018401900F08BFA70BDF0B50746F3
:105310000846584087B0C00F049048000E46590018
:1053200040084908BC1A884105D2384631461E4615
:1053300017460B4602465800400810434CD0300D2B
:10534000039040055900400D490D0590401A029008
:10535000402872DA18030121000B09050843019067
:1053600004980092002805D00199524200208841FB
:1053700000920190029840210A1A0199009800F0C9
:105380001BFA05460C466B4607CB00F036FAC019EF
:105390007141039A0E0D0023D71756401A467A40E2
:1053A000164344D0049A002A2DD0029A012A039A67
:1053B00015DC1205C01A914101263605001C714109
:1053C000D20F059ED2070093019202962A462346E9
:1053D00000F074FA07B0F0BD38463146FAE716051A
:1053E000224A0F46B218C01AB74101210905001C14
:1053F0004F4100187F41114618187941E20F1043C0
:105400006D19644113E0E2076D0815436408C20793
:105410001443039A01261205C01A91413605001C57
:105420007141CE07400830434908C01851412A460F
:10543000234600F036FACDE7FFE70498012240004A
:10544000C117121A00238B4104983146C417381A29
:10545000A141EEE730B40124E407634030BC55E7D6
:1054600030B40124E407614030BC4FE70000E0FFA6
:10547000F0B51FB488B00B990998002448400999E9
:10548000C00F490049080991C0070B9900904900D5
:1054900049080B9109990898A64608431CD00B9916
:1054A0000A98084318D0099801244000420D48008A
:1054B000410D099824050003000B204309900B9827
:1054C0000003000B20430B9050181C494018002289
:1054D00001901446104605E0002001460DB0F0BDD5
:1054E000032801DA034600E003239C46C11A0AAEF2
:1054F0000AE05F0008ADED5B4F00F75B7D430027DE
:10550000AA187C41491C5B1E6145F2DD410004ABD9
:105510005A522104120C0A43240C401C0828DFDBD9
:10552000019802900099704601910090059B049AA1
:105530000799069800F0C2F9D0E700000DFCFFFFC4
:10554000F0B50C465C4085B0E40FE40703944C00D2
:1055500000266408590094464908024602962243F0
:1055600021D062460A431ED06200570D4A000E0346
:105570002303550D012402462C492405781B1B0BDF
:10558000360B401823432643614600901C46501AB0
:10559000B44103D30098401C009002E09218009898
:1055A0005B41002803DA0020014605B0F0BD002071
:1055B000012109050746864611E064461D46141B75
:1055C000B54106D36546521BB341744607430C43AD
:1055D000A646CD0740084908284392185B41054676
:1055E0000D43EAD11046184313D060461946504087
:1055F0007140084306D06046101AB34106D201221A
:10560000002306E000220123DB0702E00122D2434F
:105610005310009874460105381C6141029C039D9B
:105620000019694100F03DF9BFE70000FD030000EB
:10563000C217C10F504010B54018CA079623002169
:1056400000F0F6F810BD10B500229623114600F0C8
:10565000EFF810BD0EB5C217C10F5040CA07401871
:105660000021054B0293019200910A460B4600F07F
:1056700025F903B000BD0000330400000EB5054954
:105680000291002100910A460B46019100F016F9A3
:1056900003B000BD33040000410040020122400A73
:1056A000D205090E80187F2901DA0020704796295B
:1056B00003DC9622511AC8407047963988407047DB
:1056C00070B5CD0F4A0009030123090B1B051943CF
:1056D0000B4BED070024520D9A4201DA002070BDF9
:1056E000074B34339A4203DC9A1A00F075F802E053
:1056F0000449511888402C43F1D0404270BD00004D
:10570000FF030000CDFBFFFF4A0009030123090B43
:105710001B051943094B10B5520D9A4201DA0020BE
:1057200010BD064B34339A4203DC9A1A00F054F849
:1057300010BD03495118884010BD0000FF03000050
:10574000CDFBFFFFC20FD207400040080BD0C10DB8
:105750000723DB01C91840020905400A1143C208AA
:10576000400711437047002001467047CB0FDB070D
:10577000490010B5490802460A4307D00A0D07241C
:105780000903E401090B121B002A01DC002010BDF3
:10579000C900440F0C43C100E018D205801800F086
:1057A0003FF810BD0122D207002800DB101A0029A3
:1057B00000DB511A8142704710B5202A04DB0146F4
:1057C000203A9140002010BD914020239C1A0346AE
:1057D000E3401943904010BD10B5202A04DB084671
:1057E000203AD040002110BD0B46D340D0402024A9
:1057F000A21A91400843194610BD10B5202A06DBB5
:10580000CB170846203A1041C1170B4306E00B4660
:105810001341D0402024A21A91400843194610BDDC
:10582000002904DA401C490001D1400840007047BB
:1058300070B40024050C05D11024000402D1002905
:1058400021D01124050E01D100020834050F01D129
:105850000001241D850F01D18000A41C002801DB5C
:105860004000641C002908D020252E1B0D46F54061
:10587000A14000D001212943084301061B1B000A57
:10588000DB1D02D5002070BC7047DB05181880189E
:105890000029F8DA401C4900F5D170BC40084000EE
:1058A000704710B5002B08DA0024401C61419218A3
:1058B0005B411A4301D14008400010BDF0B51FB450
:1058C00082B005460C0003D0084604F04BFE02E00F
:1058D00004F048FE20300246009021462846FFF79B
:1058E0006BFF049B059A04460F4618431143084377
:1058F00014D0184610431BD0009840210A1A1846AD
:105900000599FFF769FF05460E46009A0599049828
:10591000FFF752FF084305D0012004E02046394636
:1059200007B0F0BD0020C11705430E432C43374399
:1059300000990E986305401A7905E40A00220C4389
:10594000FD0A0A3002D500200146E9E701051019D9
:1059500069410C9C0D9D00196941FFF7A2FFDFE72B
:1059600010B5002904DB0124E40740428C412146A4
:10597000002B04DB1C460123DB075242A341994262
:1059800000D1904210BD0000064C0125064E05E0F6
:10599000E36807CC2B430C3C98471034B442F7D350
:1059A000FFF792FBB0B50008D0B5000838B5044643
:1059B000074908480068FFF79BFB6043009002E03E
:1059C0000098401E009000980028F9D138BD0000D2
:1059D00040420F001C01002070B5044600252068DD
:1059E00080688007800F012807D120680068C00701
:1059F000C00F002801D0012000E00020002839D18C
:105A0000206880681C490840002801D1012000E07E
:105A10000020002809D1606D102108436065A06D49
:105A200001210843A065012070BD20688068012124
:105A30000843216888600120FFF7B8FF01F05EF994
:105A400005460EE001F05AF9401B0A2809D9606D9D
:105A5000102108436065A06D01210843A065012065
:105A6000E2E720680068C007C00F012148404840B5
:105A70000028E7D00020D7E71700008010B50023EA
:105A80001A4603E0845CE3189BB2521C8A42F9D3A5
:105A9000D84380B210BD000010B5034800F028FEC6
:105AA000024800F025FE10BDC0150020781500202A
:105AB00030B51C25446C2C400125A540046C656064
:105AC000046863608468102C04D10468A2600468D0
:105AD000E16003E00468A1600468E26030BD00009A
:105AE0001449012048720A4602205E325072032097
:105AF0003C3A507204200E3A50720F480D4B007819
:105B0000087022310870203108770C495A1C087837
:105B10005871497899712333187159712033187766
:105B20005977107551751A461E32107551751076D9
:105B30005176704750110020D7000020F40000205B
:105B400010B503F0ABFE202003F054FF012005F058
:105B5000D1F8002003F04EFF044804F06FFF044822
:105B600005F01EFA002005F053FA10BDC000002019
:105B70008380000070B505200121000701F0AAF81C
:105B80000025154C002800D06560144E02213046D7
:105B900001F0A0F8002817D1012020707F20C00557
:105BA000A0600F48808F002805D0012100228902C3
:105BB000304601F09CF80B48656000880A21484394
:105BC0000949088004F020FC012000F07DFF02203C
:105BD00000F07AFF70BD00000C01002000040050AE
:105BE000500D0020E4000020F0000020704700006D
:105BF00000210A4A51610A494968012252021143AF
:105C0000074A51601146496808221143044A51600D
:105C10000021C209D201116070470000081600205F
:105C2000002002407FB500250C460646039500F093
:105C300003FFE009029003A901960095684600F071
:105C40007DFE002804D000F0BFFE002004B070BD2F
:105C500000F0BAFE0120F9E710B5002302E0C45CB1
:105C6000CC545B1C9342FAD310BD0000002039498C
:105C70008969FF2201321140914208D136494969B0
:105C800002221143344A5161FF2101310843314955
:105C90008969012252021140914208D12E49496975
:105CA000012211432C4A516101214902084329492B
:105CB0008969012292021140914208D1264949691D
:105CC00008221143244A51610121890208432149D4
:105CD00089690122D2021140914208D11E494969C5
:105CE000042211431C4A51610121C9020843194988
:105CF0008969012252031140914208D1164949692C
:105D000010221143144A51610121490308431149EA
:105D10008969012252041140914207D10E49496913
:105D2000202211430C4A5161202108430949896905
:105D3000012212041140914208D1074949694022C9
:105D40001143054A51610121090408430149886151
:105D500070470000002002400816002070B504467D
:105D600000F0CCFF05460BE0601C002808D0002C9A
:105D700004D000F0C3FF401BA04201D9032070BD36
:105D80001F488069C007C00F0028EDD11C488069FA
:105D900002210840022801D1194988611848806908
:105DA000FF2101310840884223D01548806949000D
:105DB000084088421DD01248806949000840884246
:105DC00017D00F48806949000840884211D00C481C
:105DD00080698900084088420BD009488069090120
:105DE0000840884205D0064880694910084088422A
:105DF00003D1FFF73BFF0120C1E70020BFE7000010
:105E000000200240F8B51746002605460C4600F073
:105E100013FE09E029460220226800F0E5FD002873
:105E200004D1241D2D1D361DBE42F3D300F0CCFD40
:105E3000BE4201D20020F8BD0120F8BD10B50849CE
:105E400002460020054B497905E044001C5B944262
:105E500003D0401CC0B28842F7D310BD7812002096
:105E60005800002010B500F03EFF10BD10B50948E5
:105E700001F042F980B2FFF701FC074A074BFFF738
:105E8000F7FA0022064BFFF75BFBFFF73DFC80B201
:105E900010BD000070140020F853E3A59B843E4021
:105EA00000408F4070B5384C3648217F0175617FC6
:105EB000417536490A78027649784176314905209C
:105EC000133148720A2005F05BF87D20C00005F010
:105ED00071F82C49002213310C2005F03BF9002108
:105EE0000C2005F049F9022005F09AF8284D002110
:105EF0000F2004F0C5FF2842E062F8D0E06A411CA0
:105F000030D0400430D58122D20100210F2005F08D
:105F1000F6F80021102004F0B3FF41061948490E9D
:105F20000022633004F0E2FF164D6335687A0528DD
:105F300017D102221549681DFFF744F9002810D136
:105F40001148AE7C66710422691C4030FFF716F9D7
:105F500029461331084672005130FFF70FF903202C
:105F6000207070BD02F0B2FE0A480188608B0546C1
:105F7000FFF7BEF808480088414308486D1E0180BD
:105F8000658370BDB111002058000020F40000208E
:105F900000D02724E0000020DE000020DC000020EC
:105FA00010B5084800F03AFB0A21064800F0C0FA94
:105FB000044800F06FF9800503D5024800F06DF940
:105FC00080B210BD14140020F8B52F4D002201211D
:105FD000284600F08CFEFFF7E3FFFFF734FB2B4E63
:105FE0003146FFF755F92A4C0122A0601146284698
:105FF00000F07DFE2749A068002588423EDB20781E
:10600000254F002815D02570FFF7CAFFFFF71BFBAF
:106010003146FFF73DF9A060FFF794FB00223B46B5
:10602000FFF718FA00221D4BFFF722FAFFF79EFB3D
:106030006060A068FFF786FB00223B46FFF70AFA84
:10604000174A184BFFF714FA06460F466068FFF729
:1060500079FB134A144B5242FFF70AFA32463B4689
:10606000FFF754F9FFF782FB10496060884201DDB9
:10607000616004E0FF21C905C84200D36560606823
:10608000FFF70AFBC0B2F8BD0004005000401B44FB
:10609000300000200000604000000C4000E0644040
:1060A0003333333333B33040CCCCEC3F0000C84201
:1060B000F8B5044600250026002700BF5020005DEB
:1060C000012801D10220F8BD01215020015500BF57
:1060D000206880688007800F012806D1206800684A
:1060E0000840002801D0012000E00020002841D114
:1060F000606DFF21013188430221084360652068FB
:10610000C0688707BF0F2068C068800880002168CA
:10611000C860206880680121C90708432168886039
:1061200000F0ECFD064611E000F0E8FD801B0A28B7
:106130000CD9606D0221884310210843606500BFBF
:1061400000215020015500BF0120BCE72068806875
:10615000C00FC0070121C9078842E5D02068C06888
:1061600038432168C860606D0221884301210843DB
:10617000606504E0606D202108436065012500BF73
:1061800000215020015500BF28469CE770B5044609
:106190000D4600BF5020005D012801D1022070BDD6
:1061A00001215020015500BF20688068042108406B
:1061B000800800280AD0606D20210843606500BF78
:1061C00000215020015500BF0120E8E72D496868F3
:1061D000884229D02068806A29684903490B08430E
:1061E0002168886228684003400B27490840012144
:1061F0008904884208D12548806849010843234919
:1062000088600A20FFF7D2FB28684003400B204932
:1062100008400121490488422CD11C48806849016A
:1062200008431A49886025E02068806A2968490384
:10623000490B88432168886228684003400B124953
:10624000084001218904884205D11048806849012D
:1062500088430E49886028684003400B0C49084079
:1062600001214904884205D10848806849018843D2
:106270000649886000BF00215020015500BF002062
:106280008DE70000011000000000044800270140D5
:10629000000002440146486D704701460868006CE2
:1062A0007047000010B50446002C01D1012010BD3C
:1062B000606D002806D1A0650021502001552046C0
:1062C00000F00EF9606D10210840102806D02068FB
:1062D000806804210840800800280AD0606D1021E1
:1062E0000843606500BF00215020015500BF012018
:1062F000DDE7606DFF2101318843022108436065BD
:10630000206880688007800F012807D12068006816
:10631000C007C00F002801D0012000E000200028A5
:106320003AD100BF032189076068884207D04942FB
:106330006068884203D04900606888420CD12068B8
:106340000069800080082168086120680069616830
:1063500008432168086112E0206800698000800815
:10636000216808615C4880680F21890488435A4984
:10637000886008468068616808435749886000BFA4
:106380002068C068182188432168C8602068C068F8
:10639000A16808432168C8604F4880680121490608
:1063A00088434D49886008468068A18E49060843A5
:1063B0004949886020688068012109070840002851
:1063C00004D1206880680843216888602068C0681C
:1063D000424908402168C8602169E068022901D16A
:1063E000042100E0002108432021095D49030843FE
:1063F0002C21095D49000843216B0843A1698903E9
:106400000843E169C90308432168C9680843216852
:10641000C860FF21C231606A884207D0A16A606A01
:1064200008432168C96808432168C8602120005DCD
:10643000012813D12020005D002807D12068C06802
:106440000121090408432168C86007E0606D20212C
:1064500008436065A06D01210843A065E06B012839
:1064600017D120680069FF218900884321680861ED
:10647000216C606C0843A16C0843216809690843DA
:1064800021680861206800690121084321680861CA
:106490000BE020680069C007C00F002805D0206805
:1064A0000069400840002168086120684069C00810
:1064B000C0002168486120684069A16B08432168D9
:1064C00048610020A065606D0221884301210843D6
:1064D00060650020EBE60000002701401902FEFF86
:1064E00010B586B0044614216846FEF760FE0E49DA
:1064F0002068884216D10D48416B42151143416313
:10650000C16A01221143C162C06A69461040059008
:106510000220009003200190002002900520000737
:1065200000F0E2FA06B010BD002401400010024065
:10653000F8B504460D46002600276069082801D1F9
:10654000082711E02068C068C007C00F00280AD0E3
:10655000606D20210843606500BF00215020015577
:1065600000BF0120F8BD0C2700F0C8FB064614E070
:10657000681C002811D0002D04D000F0BFFB801B48
:10658000A8420AD9606D04210843606500BF00215C
:106590005020015500BF0320E4E720680068384020
:1065A0000028E5D0606D012149020843606520683C
:1065B000C068032189020840002826D12020005D00
:1065C000002822D1206800680821084008281CD132
:1065D0002068806804210840800800280DD12068C8
:1065E00040680C21884321684860606DFF210131BB
:1065F000884301210843606507E0606D202108435E
:106600006065A06D01210843A065A069002802D142
:106610000C20216808600020A4E7000070B5044643
:1066200000252068806804210840800800282BD1BC
:1066300000BF5020005D012801D1022070BD012162
:106640005020015500BFE069012803D02046FFF724
:10665000C3F90546002D18D1606D0D490840FF2192
:106660000131084360650020A06500BF0021502073
:10667000015500BF1C202168086020688068042143
:1066800008432168886000E002252846D6E700001C
:10669000FEF1FFFF70B5044600252520005D0228AD
:1066A00003D00420E063012520E0206800680E216B
:1066B000884321680860206800684008400021681D
:1066C00008601C21606C084001218140206C416001
:1066D00001212520015500BF00212420015500BFC4
:1066E000A06B002802D02046A16B8847284670BDC9
:1066F00070B50446206C0568206806681C20616C33
:10670000014004208840284000281DD0042030404B
:10671000002819D02068006820210840002805D1F1
:106720002068006804218843216808601C21606C8F
:10673000084004218140206C4160206B00285AD021
:106740002046216B884756E01C20616C01400220E6
:1067500088402840002825D002203040002821D041
:106760002068006820210840002808D120680068BF
:106770000A218843216808600121252001551C2138
:10678000606C084002218140206C416000BF002104
:106790002420015500BFE06A00282CD02046E16A81
:1067A000884728E01C20616C014008208840284070
:1067B000002820D00820304000281CD02068006825
:1067C0000E218843216808601C21606C084001216B
:1067D0008140206C41600120E063012125200155AA
:1067E00000BF00212420015500BF606B002802D0AB
:1067F0002046616B884770BD70B50446002C01D1FE
:10680000012070BD244A2168881A1421FEF770FC0B
:10681000800060642048083820640221252001554A
:10682000206805681D480540E168A06808432169A3
:10683000084361690843A1690843E1690843216A83
:10684000084305432068056001218903A068884248
:1068500017D011487830806A1C22616C11400F22D9
:106860008A4090430C49783188621C22616C114047
:106870006068884008497831896A08430649783158
:1068800088620020E0630121252001550021242099
:1068900001550020B5E70000080002400F80FFFF0F
:1068A000F8B504460D4616461F460020009000BF6E
:1068B0002420005D012801D10220F8BD01212420FF
:1068C000015500BF2520005D01282DD10221252082
:1068D00001550020E06320680068400840002168FE
:1068E00008603B46324629462046FFF7E1F8206B18
:1068F000002806D0206800680E210843216808603F
:106900000BE0206800680421884321680860206843
:1069100000680A2108432168086020680068012196
:1069200008432168086006E000BF002124200155CB
:1069300000BF022000900098BFE70000F8B50446B1
:106940000E460127002500BF1C48007C012801D10C
:106950000220F8BD01201949087400BF1848FFF74C
:10696000FDF90746002F22D1401E3060656817E010
:106970002846FFF73DF91248FFF7F0F9074611489E
:106980004068082188430F49486008464068491517
:1069900088430C494860002F01D0356006E08035FF
:1069A000A068C00161684018A842E1D800BF00BFDC
:1069B00000200249087400BF3846CAE708160020C4
:1069C00050C30000002002400648406802210843EE
:1069D000044948600846406801210843014948606D
:1069E0000020704700200240F8B507460C461546C7
:1069F000012600BF0E48007C012801D10220F8BD0D
:106A000001200B49087400BF0A48FFF7A7F90646A2
:106A1000002E06D10649486125600648FFF79EF919
:106A2000064600BF00200249087400BF3046E6E772
:106A30000816002050C300001D484068C007C00F62
:106A4000002816D000BFEFF31080014600BF72B6D9
:106A50001848174AD0601848D06000BF81F31088EA
:106A600000BF10464068C007C00F002801D00120B9
:106A700070470F48406802221040022815D100BF1D
:106A8000EFF31080014672B60C48094A10610C48B9
:106A90001061084680F3108800BF1046406802224B
:106AA0001040022801D10120E2E70020E0E70000C9
:106AB00000200240EFCDAB8905040302BFAE9D8CE0
:106AC000161514137047000010B5044605484069B8
:106AD0002040002804D0034844612046FFF7F2FF1D
:106AE00010BD00000004014070B5034600220024E0
:106AF0000020DAE0012696400D6835402C46002C37
:106B000077D04D68022D02D04D68122D15D1D508D1
:106B1000AE001D462035A8595507EE0E0F25B5408D
:106B20000646AE4330465607F60E0D69B54028437B
:106B3000D508AD001E46203670514D68012D08D095
:106B40004D68022D05D04D68112D02D04D68122DD3
:106B500018D1986856000325B5400646AE43304626
:106B60005600CD68B5402843986058680125954087
:106B70000646AE43304610264D6835402D099540F7
:106B800028435860186856000325B5400646AE43B2
:106B900030460D79AD07AD0F5600B540284318605B
:106BA000D86856000325B5400646AE433046560029
:106BB0008D68B5402843D860012636074D683540BA
:106BC000B54271D13C4D6D6B012635433A4E75632C
:106BD0003A4D9608B600A85995072E0F0F25B540D7
:106BE0000646AE43304605252D07AB4202D10025AF
:106BF00015E059E0324DAB4201D101250FE0314D96
:106C0000AB4201D102250AE02F4DAB4201D1032551
:106C100005E02E4DAB4201D1052500E00625960783
:106C2000360FB5402843254D9608B600A851284D8B
:106C300028680546A5432846012636044D68354098
:106C4000B54202D1054625432846214D2860686893
:106C50000546A5432846012676044D683540B542D1
:106C600002D1054625432846194D6860A8680546A7
:106C7000A5432846012636054D683540B54202D168
:106C8000054625432846124DA860E8680546A543F9
:106C90002846012676054D683540B54202D10546A5
:106CA000254328460A4DE860521C0D68D540002D4A
:106CB00000D01FE770BD0000001002400800014036
:106CC0000004005000080050000C0050001C005050
:106CD00000040140024613690B40002B01D0012043
:106CE00000E00020704742694A4042617047002A34
:106CF00001D0816100E081627047000001480068B6
:106D0000704700001801002002480068401C01493B
:106D1000086070471801002010B50024084800687A
:106D20004021084306490860002000F00BF80028C5
:106D300001D0012401E000F015FA204610BD00004A
:106D40000020024070B5044600257D21C900094895
:106D50000068FEF7CDF9064601F0B8F8002801D02A
:106D6000012504E000222146501E00F01FFA2846AB
:106D700070BD00001C01002070477047F8B5394C09
:106D80000126A078401CA0702671E08A401CE08299
:106D90003548008802F0E8FD344DE888FEF753FCE2
:106DA0003349FEF775FA334F3968FEF718FA386041
:106DB0003148F105006800270090884210DB208AE6
:106DC000FEF741FC01467F20C005FEF761FA0099FD
:106DD000FEF75AFA2849086028480221017001E0AC
:106DE0002648077002212648FFF774FF002809D0C3
:106DF00027632048234A016823480091914212DD0D
:106E0000067011E0E888FEF71EFC1949FEF740FA0B
:106E1000216BFEF7E4F91D4920638842E9DB1D4937
:106E20001B48C860E5E70770688F401EFEF700FC4E
:106E30000099FEF7B7FC05D86079002802D0164803
:106E4000067001E014480770688FFEF7FCFB0949E3
:106E50000968FEF7A7FC04D26079002801D004F08D
:106E60007BFAF8BDD400002072000020500D0020F5
:106E700000007A4410010020140100206900002065
:106E8000000400500000F0425E0000200000A0401E
:106E90000400FA0500ED00E06B000020704710B51B
:106EA0000446002C01D1012010BD02212E200155E5
:106EB000204601F0E5FC204600F0F4F800212E20E9
:106EC000015500BF2D20015500BF0020ECE77047A1
:106ED000704710B5044620680068C007C00F012144
:106EE0004840484000280CD020688068084048404E
:106EF0004840002805D00120216848602046FFF75F
:106F00003DFF2068006802210840400800280BD09F
:106F10002068806808404008002805D002202168C9
:106F200048602046FFF728FF2068006804210840D9
:106F3000800800280BD0206880680840800800285E
:106F400005D0042021684860204600F009F9206837
:106F5000006808210840C00800280BD0206880681D
:106F60000840C008002805D0082021684860204655
:106F7000FFF794FF206800681021084000090028EE
:106F80000BD02068806808400009002805D0102038
:106F9000216848602046FFF7F0FE20680068202145
:106FA0000840400900280BD020688068084040094C
:106FB000002805D02020216848602046FFF788FF80
:106FC0002068006840210840800900280BD0206814
:106FD000806808408009002805D04020216848606A
:106FE0002046FFF774FF10BD70B50446002C01D198
:106FF000012070BD6068012800D100BF264960698A
:10700000884200D000BF2E20005D002805D100215D
:107010002D200155204600F057F802212E20015561
:107020002068C5686068012803D08905A06A884285
:1070300003D11E21284688430546174960698842C6
:1070400001D01648054016480540A168606808430D
:10705000216A0843616A0843A16A084305436068DE
:10706000012804D00121C905A06A884203D1E16842
:1070700020690843054308496069884205D0616971
:10708000A0690843E169084305432068C560012100
:107090002E2001550020ACE7FFFF00003F1FFFFF3F
:1070A000F8F119FF10B500680549884207D1054875
:1070B000816B4900490881630D2000F05FF810BD25
:1070C000007C00400010024010B50068084988426A
:1070D0000CD10848816BC204114381630022012155
:1070E0000D2000F063F80D2000F054F810BD0000F2
:1070F000007C00400010024001460868C0697047EB
:1071000010B5034602242E20C454144800682407F6
:107110002043124C20601868C0680124E404204316
:107120001C68E06018688068012420431C68A06027
:1071300018680069012420431C6820611868816177
:107140001868426118680069042420431C682061A3
:1071500001242E20C454002010BD00000004014072
:10716000704700000448416B012211434163816B69
:1071700002041143816370470010024000BFC20641
:10718000D20E01219140024A116000BF70470000F9
:1071900080E100E000BFC206D20E01219140024A08
:1071A000116000BF7047000000E100E070B50446C8
:1071B0000D4616462946204601F04CFD70BD0000E4
:1071C000024949688143014A51607047007000409C
:1071D00003480068FF2101310843014908607047F6
:1071E00000700040024949680143014A51607047FC
:1071F0000070004007480068022108430549086004
:1072000005480069042108430349086100BF00BF25
:1072100030BF70470070004000ED00E010B502463E
:1072200000200E4B18688008800003461343184660
:107230000A4B18600A4B1B6904242343084C236142
:10724000012901D130BF02E040BF20BF20BF044B65
:107250001B690424A343024C236110BD007000404D
:1072600000ED00E0F8B50446202120680840202801
:107270007CD120680840202800D100BF0027814829
:10728000806B012109070840002805D17D48806BEB
:1072900008437C49886301277B480068FF2101314E
:1072A0000840002816D178480068084376490860ED
:1072B000FFF724FD064606E0FFF720FD801B64284B
:1072C00001D90320F8BD70480068FF210131084052
:1072D0000028F1D06B480568032109050D4060685E
:1072E0000840A8420DD0091160680840884208D1C2
:1072F00064480068012149040840884201D1012006
:10730000E0E7604840300069032109040840054671
:10731000002D3DD060680840A84239D02021206867
:107320000840202834D1574840300069032109041F
:10733000884305465348403000690121C904084389
:10734000504940310861084600690121C904884359
:107350004C4940310861084605618015284089156F
:10736000884215D1FFF7CAFC064608E039E0FFF76E
:10737000C5FC801B4549884201D90320A2E741484A
:1073800040300069012149020840400A0028EED03F
:1073900000BF00BF032109046068084088420AD189
:1073A00038480068090188430322120561681140CA
:1073B00008433449086000BF324840300069032266
:1073C00012046168114008432E494031086100BF32
:1073D000012F05D12B48806B890588432949886393
:1073E00000BF2078C007C00F002809D025484030D2
:1073F000C06880088000A168084322494031C86005
:10740000022120680840022809D11E484030C06887
:107410000C218843E16808431A494031C8600421BF
:107420002068084004280AD116484030C06803216B
:10743000890288432169084312494031C860082104
:107440002068084008280AD10E484030C06803214F
:1074500009038843616908430A494031C8608021B3
:107460002068084080280AD106484030C0680321BF
:1074700089048843A169084302494031C86000205B
:1074800020E7000000100240007000408813000058
:10749000F8B504460D46002C01D10120F8BD79480D
:1074A0000068C007C00FA8420ED2764800684008A6
:1074B000400028437349086008460068C007C00FB1
:1074C000A84201D00120E9E70221206808400228F3
:1074D00007D16D48C068F0218843A16808436A4914
:1074E000C8602078C007C00F00284CD06068022810
:1074F00009D165480068012149040840400C002872
:1075000024D10120CAE76068032809D15E480068D9
:10751000012149060840400E002817D10120BDE78F
:107520006068012808D15848006804210840800894
:1075300000280BD10120B1E753480068012149021E
:107540000840400A002801D10120A7E74E48C06842
:1075500080088000616808434B49C860FFF7CEFB94
:107560000646606802280FD107E0FFF7C7FB801BC3
:107570004649884201D9032090E74348C0680C215E
:1075800008400828F1D134E0606803280FD107E0F3
:10759000FFF7B4FB801B3D49884201D903207DE7FA
:1075A0003948C0680C2108400C28F1D121E06068FE
:1075B00001280FD107E0FFF7A1FB801B3349884268
:1075C00001D903206AE73048C0680C21084004282C
:1075D000F1D10EE007E0FFF791FB801B2B498842B9
:1075E00001D903205AE72848C0680C210840002828
:1075F000F1D124480068C007C00FA8420ED9214825
:1076000000684008400028431E490860084600689A
:10761000C007C00FA84201D001203FE70421206825
:107620000840042808D11848C06807210902884387
:10763000E16808431449C860082120680840082808
:1076400009D11148C0680721C90288432169C900CE
:1076500008430D49C86000F049F80B49C968F02299
:10766000114009090A4A515CC8400A4908600020D3
:10767000FFF768FB0746002F01D038460EE70020D1
:107680000CE70000002002400010024088130000B8
:107690008EB500081C0100200148006870470000FA
:1076A0001C01002000B5FFF7F7FF0549C968072254
:1076B00012021140090A034A515CC84000BD000093
:1076C000001002409EB5000800B5FFF7E5FF054930
:1076D000C9680722D2021140C90A034A515CC84056
:1076E00000BD0000001002409EB50008FEB52E4807
:1076F000C7680C203840002845D0042804D008284A
:107700000CD00C283ED10BE027480068102108401F
:10771000002801D0254C00E0254C41E0254C3FE0FD
:107720000F2080043840800C23490E5C0320800524
:107730003840800D401C01901B48C068012109049D
:107740000840002807D01B49714308460199FDF7FE
:10775000CFFC054614E014480068102108400028BA
:1077600007D01249714308460199FDF7C1FC05464F
:1077700006E00F49714308460199FDF7B9FC05463B
:107780002C460DE000BF0848406807214903084027
:10779000400B00900098401C01218140CC0300BFA9
:1077A00000BF2046FEBD00000010024000093D0061
:1077B0000024F40000127A00A6B50008FEB50446C5
:1077C000002C01D10120FEBDF848C6680C210E40F6
:1077D000C768012109040F402078C007C00F0028A6
:1077E00072D0082E04D00C2E0FD1084687420CD13F
:1077F000EE480068012149040840400C002863D08D
:107800006068002860D10120DDE700BF0121090484
:107810006068884205D1E54800680843E34908608C
:1078200027E005210904606888420ED1DF4800681E
:10783000012189040843DD490860084600680121E8
:1078400009040843D949086013E0D84800680121B9
:1078500009048843D54908600846006801210904E5
:107860000840009000BFD148006889008843CF4994
:10787000086000BF6068002813D0FFF73FFA054694
:1078800006E0FFF73BFA401B642801D903209AE782
:10789000C6480068012149040840400C0028F0D087
:1078A00012E0FFF72BFA054606E0FFF727FA401B28
:1078B000642801D9032086E7BC48006801214904F7
:1078C0000840400C0028F0D102212068084002281E
:1078D0007AD1E0680290042E03D00C2E34D1002F10
:1078E00032D1B2480068042108408008002804D042
:1078F0000298002801D1012065E7AC4840681F21AB
:1079000009028843216909020843A84948600846DA
:1079100000680921884302990843A4490860FFF7D9
:10792000E5FEA249C968F02211400909A04A515C4C
:10793000C840A04908600020FFF704FA01900198B0
:10794000002841D001983EE70298002824D09748AB
:107950000068092188430299084394490860FFF7A9
:10796000CDF9054606E0FFF7C9F9401B022801D909
:10797000032028E78D48006804210840800800287B
:10798000F1D08A4840681F21090288432169090211
:1079900008438649486017E0844800684008400072
:1079A00082490860FFF7AAF9054606E0FFF7A6F945
:1079B000401B022801D9032005E77C480068042108
:1079C000084080080028F1D11021206808401028C4
:1079D00067D1002E36D17548006849010840400A39
:1079E000002804D0A069002801D10120EBE66F48EF
:1079F0004068072149038843216A08436B4948606E
:107A0000084640680002000A217F090608436749CA
:107A10004860206A400B401C01218140C803634933
:107A2000C968F02211400909614A515CC8406149A6
:107A300008600020FFF786F90190019800284BD0DC
:107A40000198C0E6A06900282CD058480068FF21A2
:107A50000131084355490860FFF750F9054606E033
:107A6000FFF74CF9401B022801D90320ABE64F4831
:107A70000068012149020840400A0028F0D04B4824
:107A80004068072149038843216A08434749486001
:107A9000084640680002000A217F0906084343495E
:107AA000486019E041480068FF21013188433F499F
:107AB0000860FFF723F9054606E0FFF71FF9401BB2
:107AC000022801D903207EE63848006801214902D6
:107AD0000840400A0028F0D1082120680840082802
:107AE00039D1606900281BD030484030006901213D
:107AF00008432E4940310861FFF700F9054606E0CA
:107B0000FFF7FCF8401B022801D903205BE6274859
:107B1000403000690221084040080028F0D01AE0F7
:107B20002248403000694008400020494031086147
:107B3000FFF7E4F8054606E0FFF7E0F8401B0228EF
:107B400001D903203FE6194840300069022108406E
:107B500040080028F0D1042120680840042879D189
:107B6000002000901148806B89060840002806D14B
:107B70000E48806B08430D498863012000900E4831
:107B80000068FF210131084000281ED10A48006822
:107B9000084309490860FFF7B1F805460EE0FFF712
:107BA000ADF8401B642809D903200CE60010024000
:107BB0008EB500081C010020007000408548006858
:107BC000FF21013108400028E9D000BFFF21013129
:107BD000A068884205D18048006908437E49086151
:107BE00030E0A06800280DD17B480069FF210131F9
:107BF0008843794908610846006909158843764930
:107C000008611FE005210902A06888420DD1724871
:107C100000690121890208436F490861084600692B
:107C2000891508436C4908610CE06B480069FF2125
:107C3000013188436849086108460069091588438D
:107C40006549086100BFA068002815D0FFF756F805
:107C5000054608E031E0FFF751F8401B5F498842D4
:107C600001D90320AFE55C480069012149020840C1
:107C7000400A0028EFD013E0FFF740F8054607E080
:107C8000FFF73CF8401B5549884201D903209AE58B
:107C900051480069012149020840400A0028EFD1FB
:107CA0000098012808D14C484038806B0121090711
:107CB000884349494039886300BF606A00284CD036
:107CC0000C2E69D0606A022848D1434840380068C9
:107CD000012109068843404940390860FFF70EF842
:107CE000054606E0FFF70AF8401B022801D90320E9
:107CF00069E5394840380068012149060840400ECE
:107D00000028EFD1E16AA06A0843216B0843324999
:107D10004039C968FD221204914308432E49403975
:107D2000C860084600680121090608432A4940390D
:107D30000860FEF7E3FF054606E0FEF7DFFF401BA5
:107D4000022801D903203EE523484038006801217C
:107D500049060840400E0028EFD038E01E48403861
:107D600000680121090688431B4940390860FEF775
:107D7000C5FF054606E0FEF7C1FF401B022801D9FA
:107D8000032020E5144840380068012149060840D6
:107D9000400E0028EFD11AE0606A012800D112E5F8
:107DA0000D484038C768012000043840A16A884265
:107DB0000BD10F2080043840E16A884205D10320AE
:107DC00080053840216B884201D00120FBE400206F
:107DD000F9E40000007000404010024088130000E9
:107DE00010B50446002C01D1012010BD606A0028A6
:107DF00000D100BF0021A1625120005D002804D104
:107E000050200155204600F035F80221512001553F
:107E1000206800684021884321680860A168606884
:107E20000843E16808432169084361690843012266
:107E30005202A16911400843E1690843216A0843DD
:107E4000A16A084321680860A069000C0421084069
:107E5000616A0843216848602068C06991008843CE
:107E60002168C86100206065012151200155002072
:107E7000BBE7000010B586B0044614216846FDF744
:107E800096F910492068884219D10F48416B821435
:107E900011434163C16A01221143C162C06A0021DA
:107EA00010400590E02000900220019003200390F4
:107EB00002910491052069460007FEF715FE06B001
:107EC00010BD0000003001400010024070B50446B3
:107ED0002546681E0949884201D901200CE0681E28
:107EE000074948610321081F00F0B4FE002004493F
:107EF000886107200861002070BD0000FFFFFF00BF
:107F000000E000E070477047FEB504462068C56990
:107F100020680668206887682807000F019001988C
:107F200000280ED12020284000280AD020203040F0
:107F3000002806D0206E002802D02046216E8847F7
:107F4000FEBD019800287DD0F807C00F002804D19D
:107F5000FF20213030400028F5D0E807C00F00286E
:107F60000BD0FF2001303040002806D001202168CE
:107F70000862E06F01210843E067022028400028E2
:107F80000AD0F807C00F002806D002202168086236
:107F9000E06F04210843E0670420284000280AD04D
:107FA000F807C00F002806D0042021680862E06F9F
:107FB00002210843E0670820284000280ED0202036
:107FC0003040002803D1F807C00F002806D0082051
:107FD00021680862E06F08210843E067E06F00282D
:107FE00046D020202840002809D0202030400028FA
:107FF00005D0206E002802D02046216E8847E06F11
:1080000000902068806840210840402804D0082162
:1080100000980840002826D0204601F062FF206822
:10802000806840210840402819D120688068884332
:1080300021688860E06E00280DD02548E16E8863D5
:10804000E06E00E015E0FEF725FB002810D0E06EA2
:10805000816B88470CE02046FFF755FF08E020467B
:10806000FFF751FF04E02046FFF74DFF0020E067D7
:1080700066E701200005284000280CD0012080057B
:108080003840002807D001200005216808622046FA
:10809000FFF738FF54E78020284000280AD08020CE
:1080A0003040002806D0606E002802D02046616E65
:1080B000884745E740202840002807D0402030402E
:1080C000002803D0204601F01EFF39E700BF37E744
:1080D000219E000810B50446002C01D1012010BDDE
:1080E000A069002800D000E000BF606F002805D123
:1080F000002170200155204600F02CF824206067F4
:10810000206800684008400021680860204601F0AF
:1081100045FF012800D1E2E7606A002802D020462E
:1081200001F046FD206840680921C90288432168A2
:108130004860206880682A21884321688860206818
:1081400000680121084321680860204601F0A8FD6D
:10815000C5E70000F0B587B0064614216846FDF774
:1081600026F82C493068884251D12B48416B0122B6
:10817000920311434163C16A01221143C162C06A83
:1081800000251040059003204002009002200327A4
:1081900001A9A1C104200490052069460007FEF74B
:1081A000A3FC1F4C1D48A560E56081C48027E560E5
:1081B000A7602020256160610002A0611848083C8A
:1081C000FEF71AFB002801D0FDF710FDF466A66249
:1081D000144C12482146143820600320606010209F
:1081E0000831A1C16561A561E56120462562FEF700
:1081F00003FB002801D0FDF7F9FCB4660022012141
:108200001B20A662FEF7D2FF1B20FEF7C3FF07B0BC
:10821000F0BD000000380140001002403000024074
:1082200078150020C015002070B504460D4616468E
:10823000A06F202863D1002D01D0002E01D1012094
:1082400070BD01210903A068884208D12069002877
:1082500005D1E807C00F002801D00120F0E700BFDA
:108260007020005D012801D10220E9E70121702082
:10827000015500BF6565582006530020E0672220A5
:10828000A067E06E002820D01E48E16EC8621E483C
:10829000E16E08631D48E16E48630020E16E88636B
:1082A0002368194624313346626DE06EFEF7F8FA12
:1082B00000280AD01020E06700BF0021702001557F
:1082C00000BF202060670120BAE700BF00217020B6
:1082D000015500BF20680068FF2101310843216873
:1082E0000860206880680121084321688860206850
:1082F000806840210843216888600020A0E70220B0
:108300009EE700008B9E0008D59E0008399E00085D
:1083100070477047FFB583B004460D461746606F3F
:10832000202875D1002D01D0002F02D1012007B0E7
:10833000F0BD01210903A068884208D12069002806
:1083400005D1E807C00F002801D00120EFE700BFEA
:108350007020005D012801D10220E8E70121702092
:10836000015500BF0020E06721206067FEF7C6FCD2
:108370000190502007535220075301210903A068A0
:10838000884205D12069002802D10026029502E02A
:108390002E460020029021E00698009000228021C5
:1083A0002046019B01F0E8FF002801D00320BEE732
:1083B000002E09D102980088C005C00D216888628E
:1083C0000298801C029003E0307821688862761C55
:1083D0005220005B401E81B2522001535220005BAC
:1083E0000028D9D106980090002240212046019B08
:1083F00001F0C2FF002801D0032098E72020606729
:1084000000BF00217020015500BF00208FE7FFE76B
:1084100002208CE77047000001490248C160FDE777
:108420000400FA0500ED00E010B505242407002241
:1084300004212046FEF75BFC002208212046FEF7BF
:1084400056FC0A2002F0B3FA012204212046FEF76E
:108450004EFC0A2002F0ABFA002204212046FEF76F
:1084600046FC10BD10B50524240700220421204637
:10847000FEF73DFC012208212046FEF738FC0A20C9
:1084800002F095FA012204212046FEF730FC0A2072
:1084900002F08DFA002204212046FEF728FC10BDD0
:1084A000F8B5002405260746254636070022042194
:1084B0003046FEF71CFC0A2002F079FA0122042162
:1084C0003046FEF714FC6006040E08213046FEF725
:1084D00001FC002801D0641CE4B2052002F067FA18
:1084E0006D1CEDB2082DE1D3002F03D0FFF79CFFE8
:1084F0002046F8BDFFF7B6FFFAE770B5052605463A
:108500003607002204213046FEF7F1FB0024E8097B
:1085100001D0012200E0002208213046FEF7E7FBEF
:108520006806050E0A2002F042FA012204213046B4
:10853000FEF7DDFB0A2002F03AFA00220421304661
:10854000FEF7D5FB0A2002F032FA641CE4B2082CD4
:10855000DDD370BD10B50524240701220821204673
:10856000FEF7C5FB012204212046FEF7C0FB0022D6
:1085700008212046FEF7BBFB0A2002F018FA002271
:1085800004212046FEF7B3FB10BD10B505242407D7
:10859000002204212046FEF7AAFB002208212046E3
:1085A000FEF7A5FB0A2002F002FA01220421204670
:1085B000FEF79DFB012208212046FEF798FB0A20CA
:1085C00002F0F5F910BD70B505252D070024012234
:1085D00008212846FEF78BFB062002F0E8F901226D
:1085E00004212846FEF783FB062002F0E0F907E0AD
:1085F000641CE4B2FA2C03D9FFF7C7FF012070BD59
:1086000008212846FEF766FB0028F1D1002204214C
:108610002846FEF76CFB002070BD0000F8B501F0A5
:1086200077FB01F0B1FB47480068C069464E474FF1
:10863000800700D5FE60FDF719FC4549454C898F40
:10864000002914D044490A7801218902002A0AD05D
:10865000012A04D0022A04D0032A08D103E02128E9
:1086600001D2002200E001222046FEF740FB01215A
:10867000C9023848FEF72EFB384C0025002824D0CC
:1086800037480560E079002803D10120E07101F04E
:10869000BBFE2078632806D9002208212D48FEF76A
:1086A00026FB012205E0012208212A48FEF71FFBD4
:1086B000002201210520C9030007FEF718FB244C06
:1086C0004034A08C012803D01CE0E5710022EBE7C8
:1086D00024486946088072B680212348FDF7A2FA33
:1086E000002804D0022269461F48FDF78BFB62B6C2
:1086F0001EA001F027FFA58402F0CAFE642002F04C
:108700004FF9FE60608C012808D11148658405800E
:1087100002F0BEFE642002F043F9FE60208C0128C6
:1087200006D1258402F0B4FE642002F039F9FE601F
:108730000748124A0188914202D1C088002800D11E
:10874000FE60F8BDF81400200400FA0500ED00E01A
:10875000500D00200004005069000020D4000020CB
:1087600010010020AAAA0000384A0008BDF8C8EB92
:10877000C9FDBCB6C4A3CABD0D0A0000AA550000BD
:1087800008B53721202000F06EF80321212000F0E9
:108790006AF84021222000F066F80821232000F02A
:1087A00062F8AA21302000F05EF80A48008FC1B2BA
:1087B000322000F058F80221332000F054F85F21F5
:1087C000202000F050F8684600F006F80A2002F079
:1087D000EEF808BD500D002010B501460F2000F046
:1087E00021F8002800D0012010BD10B50446FFF785
:1087F000B1FE3220FFF781FEFFF7E5FEE0B2FFF7A2
:108800007CFEFFF7E0FEFFF7A5FE3320FFF775FEC5
:10881000FFF7D9FE0020FFF743FE0446FFF7B5FE41
:10882000204610BD10B50C46FFF7DFFF2070012079
:1088300010BD70B50D460446FFF78CFE3220FFF7E1
:108840005CFEFFF7C0FEE0B2FFF757FEFFF7BBFE8E
:108850002846FFF752FEFFF7B6FEFFF796FE0A2006
:1088600002F0A5F870BD10B5FFF7E3FF012010BDC1
:1088700010B50248FEF72DFB10BD0000701400205B
:10888000F0B585B004460020039072B64F492068C9
:108890004018002806D14E48C068032189040840CA
:1088A000039000E000BF00BF20688068029020684D
:1088B000C06801902068456920688669434920683E
:1088C000401800280DD142484038806A49050843C5
:1088D0003F49403988620846806A40004008886203
:1088E00000E000BF00BF002D01D1002E5FD037494E
:1088F00020684018002807D13548C0680321890442
:1089000088433349C86000E000BF00BF002D1DD080
:1089100020680069012108432168086120684561D9
:10892000FEF7ECF9074600BFFEF7E8F9C01B009020
:108930002068006808210840082804D07D21C9006B
:1089400000988842F0D9082021684860002E1DD088
:108950002068006901210843216808612068866158
:10896000FEF7CCF9074600BFFEF7C8F9C01B009020
:108970002068006810210840102804D07D21C9001B
:1089800000988842F0D91020216848600F4920687B
:108990004018002809D10E48C06803218904884383
:1089A000039908430A49C86000E000BF00BF20687F
:1089B00000694008400021680861029821688860C9
:1089C00001982168C86062B605B0F0BD0084FFBFA1
:1089D000401002401CB5002116480091144A019134
:1089E0000260C16312054260816007228263012236
:1089F00002610246C16020321170FF235170C23300
:108A000043628162117301638161042241634261A7
:108A1000C161FDF747FC084800908013019069464A
:108A20000448FDF7B3FB00210248FDF741FB1CBDE4
:108A300000240140141400200200000408B5084876
:108A4000016B012211430163006B01211040009072
:108A500000220A20FEF7AAFB0A20FEF79BFB08BDB6
:108A600000100240F0B587B014216846FCF79FFB68
:108A70004C48C26A04210A43C262C26A0A40059293
:108A8000C16A80273943C162C16A39400591C16A10
:108A900001252943C162C16A29400591C16A0226A4
:108AA0003143C162C06A2A463040059005201C212E
:108AB0000007FEF71CF901223B493C48FEF717F975
:108AC00000223B493948FEF712F991210520002286
:108AD00009020007FEF70BF9364801900024052033
:108AE0006946009502940007FDF7FEFF0320019000
:108AF00005206946009602940007FDF7F5FF0C205B
:108B000000901120019003200390052002946946F3
:108B10000007FDF7E9FF1020009005206946039645
:108B2000019502940007FDF7DFFF112001900294E8
:108B30006946009503941D48FDF7D6FF1E48019035
:108B40006946009602951948FDF7CEFF1B48009034
:108B500002946946019503941448FDF7C5FFE802A5
:108B60006A4651C269461148FDF7BEFF91200002D6
:108B70000090052002946946019503940007FDF7D3
:108B8000B3FF69460948009702950194FDF7ACFFD1
:108B9000002201210520FEF709FB0520FEF7FAFA65
:108BA00007B0F0BD001002400106000000040050B4
:108BB00008300000000011100000211008360000ED
:108BC00010B50F4C0D482060FF200530606000207C
:108BD000A060E06020616061E061012120624902E3
:108BE0006062A161A0620720E0622046FFF7F8F80A
:108BF0002068016840221143016010BD003001402F
:108C0000A014002000B585B014216846FCF7CFFA07
:108C10000E480D490160E121490241600021816057
:108C2000C160016181610C22C16142610162302138
:108C300041620121090381634900C163FFF74AFAD8
:108C400001F0DCFB05B000BD00380140F814002045
:108C50007047000010B5002819DA1A4A03071B0FE5
:108C6000083B9B089B00D2588307DC0EFF23A340E0
:108C70009A438B071B0E8407E40EA3401A43114B43
:108C80000407240F083CA408A4001A5118E00E4A57
:108C900003231B02D21883089B00D2588307DC0EE3
:108CA000FF23A3409A438B071B0E8407E40EA340C7
:108CB0001A43054B032424021B198408A4001A51EB
:108CC00010BD00001CED00E000E100E0BFF34F8F9D
:108CD00004490348C860BFF34F8F00BFFDE70000A1
:108CE0000400FA0500ED00E0F0B587B00A2002F0BC
:108CF00047F97D20C00002F05DF9F94C0025A57010
:108D0000607B0C2801D30B206073012205205102E7
:108D10000007FDF7ECFF0026F248E670F24D007800
:108D20002871F249A079097840000843E17C890064
:108D30000843E871A06AE870401CA0626079294687
:108D4000A8744200B4310846A138FCF717FA06208F
:108D50006872E74829460078A872A07E2873133904
:108D6000207F0875607F48756079002240001331CC
:108D7000153002F0EFF9607900214000153002F063
:108D8000FBF9022002F04CF9EE71E673A6720125A0
:108D90002573E672D748FEF7AFF920840746E670E0
:108DA0006079FCF76BFCD44AD44BFCF761FB01F013
:108DB00093FD0022AB07FCF7A9FAFCF7A5FC00061F
:108DC000C10CC81980B2E9036084884201D3401AFB
:108DD0006084CB4860632079401C2071C548FEF751
:108DE0008BF9E083C0480C30064642364030039091
:108DF000ABE1C048FEF780F9E083C24F0BE0BD480D
:108E0000FEF77AF980B2E083618C884203D3BE4AD0
:108E10008918884206D300210F2002F031F8384229
:108E2000E062ECD0E06A411C21D040047ED5812272
:108E3000D20100210F2002F062F97D20C00002F073
:108E4000B9F8002002F06BF80021102002F018F8A9
:108E50004106A548490E274600225030616402F0C1
:108E600045F8A1485030417A0729C1D101E0FFF708
:108E70002DFF0222A549401DFCF7A4F90028B7D117
:108E800002F0CBF979653C46386502F0B3F9F96533
:108E9000B865F8786A46401CF87093484D300179FF
:108EA00011704079507010880090B98B884273D14E
:108EB0009749308A08800398808A20838D48FEF77E
:108EC0001BF9E08301F0EEFEFF23A26D5B04E06D71
:108ED0000021D21848410006170A074379084900C3
:108EE000080E0902216660667F48636D0A30226DB4
:108EF00002F068F96079E36D81007B48A26D081883
:108F0000163002F05FF97848636E1230226E02F07C
:108F100059F9754808214172607900228000724930
:108F20001C3002F017F96079800000E000E10021B8
:108F30001C3002F021F9384602F01BF8012002F043
:108F40006FF8207202217348FDF7C4FE002824D078
:108F500000216648624A0170B1891186F089508605
:108F6000614F226B50376263FB7C1A07120F032A92
:108F700000D062741A090026A2742671584BA5729B
:108F80009986D886002A17D002226049781DFCF7FE
:108F900019F9002803D00FE076E00121D9E7524803
:108FA000E573C571606C50491638C2B26631084627
:108FB0002274D230FCF7E2F8E572208B5649FF307C
:108FC000C33080B2208388420CD9494240182083A4
:108FD0004F487D220188D200491C89B2018091420C
:108FE00000D306804A48218B06887D20C00070434C
:108FF0004018A06306904948302107784848A77375
:1090000000884843FCF71FFB00900A207043FCF7E0
:109010001AFB0099FCF73CF97F21C905FCF7DFF842
:10902000FCF73AFB80B23D497F1E0880B84200D170
:10903000E572A6841420205EFCF70CFB06460F4662
:10904000E08BFCF71BFB374A374BFCF711FA049017
:1090500005910698FCF7FEFA059B049AFCF7FAF9CD
:1090600032463B46FCF752F9FCF72AFBE063608B83
:1090700000F07AFC207A002870D100210F2001F046
:10908000FFFE0006F9D569E0FCF7D8FE274A032168
:1090900011541349B28987000A862448F2894A8606
:1090A000603839180398008B08802049206B3039CC
:1090B000C8510D48E36D38181630A26D02F082F8E1
:1090C0001A486038C159206B81423EDD00293CD0EE
:1090D0002146002839D0009888830220207034E08F
:1090E00058000020D4000020C41100200C010020F2
:1090F000E400002070140020B81E85EB51B8CE3F6C
:10910000A086010000D02724983A0000F400002037
:109110000801002000040050E7030000EA000020DE
:10912000EE000020F853E3A59B843E40F01200209F
:109130003A4600210F2001F0E2FF6079E178401CFF
:10914000814202D0002001F0EAFEE18B608C814276
:1091500000D24EE6184A80188142FAD801F0A2FDEA
:10916000164A00210F2001F0CAFF20790A2800D9F1
:109170002570E07B002805D011490B7848788A7863
:10918000022B0ED00D4A002180320F2001F0B7FFD4
:1091900001210520002249020007FDF7A8FD07B0C4
:1091A000F0BD084BC91C1818FBF7E8FF02F070F976
:1091B000642001F0F5FB5AE6983A000000D027241D
:1091C000FC120020500D002070470000F0B58DB05B
:1091D000B54801900020C0430A9000260A2001F003
:1091E000CFFE7D20C00001F0E5FE0020AF4C05461B
:1091F000A070AF4FAF480B90AE480022C2388573C5
:109200000146142001F0A6FF0021142001F0B4FF54
:10921000022001F005FF00210F2001F031FE38424D
:10922000E062F8D0E06A0146401C18D048047DD5C1
:109230008122D20100210F2001F061FF00211020C6
:1092400001F01EFE41069B48490E0022801C01F0E1
:109250004DFE9848801C417A022902D004E1FFF7B4
:1092600035FD944802229449C01DFBF7ABFF00284E
:10927000F4D101F0D2FF6165206501F0BBFFE1652B
:10928000A065002E22D10B988C49008A088089485D
:109290000126801E808A20838948FDF72DFFE08308
:1092A000208B8849FF30C33080B2208388420DD99B
:1092B00049424018814920830888824A401C80B274
:1092C0000B320880904201D3002008800B98694639
:1092D00082890A80C089488076490422C91C0846D0
:1092E000A238FBF74BFFFF22A16D5204E06D002373
:1092F000891858410006090A01430846029101F005
:1093000038FE029948084000010E0002616620669E
:109310006848636D9638226D01F054FF6548E36D2F
:109320009238A26D01F04EFF624800E09EE08E3858
:10933000636E226E01F046FF5E490022A0393C2098
:1093400001F008FF00213C2001F016FF012001F090
:1093500067FE2072A0780121401CA0700520C9037F
:109360000007FCF77FFD55487D220088D2000146AA
:1093700002905043228B0A398018A0630C90524807
:109380000078A073049008B2E084002803DA7D21FD
:10939000C9004018E0844D48302100884843FCF75C
:1093A00052F905902620205EFCF742F90599FBF75B
:1093B0006FFF7F21C905FBF712FFFCF76DF94249EA
:1093C00080B208800499491E884201D10120E072D0
:1093D0000298A0841420205EFCF73CF905910690C9
:1093E000E08BFCF74BF93A4A3A4BFCF741F807910E
:1093F00004900C98FCF72EF9079B049AFCF72AF8C6
:10940000059B069AFBF782FFFCF75AF9E063608B35
:1094100000F0AAFA0099019881420DDA00290BD0D8
:1094200024490422C91C0AA8FBF7A8FE02202070C8
:109430000520607200980190207A002805D1002153
:109440000F2001F01DFD0006F9D5802200210F201C
:1094500001F055FE00206D1CEDB26070032D00D2AE
:10946000CAE6002E08D01AE00120F4E71A4A0021CB
:109470000F2001F044FEF7E7608B401E0104090C49
:109480001648618302D00288914201D90088608326
:109490001349608B0988401E4843124908800A9886
:1094A000A0830DB0F0BD00003F420F005800002027
:1094B00000D0272412120020F40000200801002010
:1094C00070140020E7030000EA000020EE000020F6
:1094D000F853E3A59B843E4000902724E000002041
:1094E000DE000020DC000020F8B531492F4808607C
:1094F00001F06EFF304C2F486080E088002801D1D9
:109500006420E080208F0A2801D902202087E08E85
:109510003C2801D93C20E086284980B20870284DBB
:10952000E08F6871A08FA871A07AE870A6880521E5
:109530002E626981E7883846FBF7DAFDA88101468B
:109540003046FBF7D5FD8800081886B27D20C000A4
:109550002E817043FCF792F81A4A1B4BFBF7F0FF81
:10956000FCF7D2F8E8817D206E823946C000FBF717
:10957000BFFD28820146C820FBF7BAFD68830120A1
:10958000E882FCF773FCA882EA8910491048FDF7CD
:10959000B7FD10A0296A00F0D5FFE18811A000F006
:1095A000D1FF218914A000F0CDFFF8BD35A400083B
:1095B0005000002009020000500D00200000002093
:1095C000D4000020F853E3A59B843E40FF7F0000B9
:1095D00070140020B1EAC7A949443A202564202E1E
:1095E0000D0A0000CDA8D1B6BCE4B8F43A20256439
:1095F000206D732E0D0A0000B5A5B4CECDA8D1B64E
:10960000BBF9D5BECAFDC1BF3A202564B8F62E0D00
:109610000A000000F0B5904D85B0012028808F4FE2
:10962000C8208F4C3880E079401CE071C00706D01C
:10963000608B411E6183022801D2C8206083608B49
:1096400000F092F90A2001F09BFC7D20C00001F09F
:10965000B1FC02218348FDF73DFB002838D00020F3
:10966000814980000978824E490008437F49097882
:109670000843B072102070727E48C1887D20C000FF
:10968000FBF736FD70737C487A490078B07330463A
:109690000B308A780270C9784170411C75482030BF
:1096A000027ECA70407E087172482230027E4A7182
:1096B000407E887100220C39152001F04BFD0021FD
:1096C000152001F059FD022001F0AAFC6B4E03E0C9
:1096D0000120C5E7FEF7A2FF00210F2001F0D0FB1B
:1096E0003042E062F6D0E06A411C7DD040047CD577
:1096F0008122D20100210F2001F001FD0021102064
:1097000001F0BEFB41065A48490E00225030616408
:1097100001F0ECFB564E5036707A112865D10222CA
:109720005749701DFBF74EFD00285ED1F01E0279EF
:1097300069460A7040794870B17A2980C820FBF7E1
:10974000D7FC3880307B60834E4DB01E008A288065
:10975000301F808A20834C48FDF7CEFC80B2E08326
:109760000390208B4949FF30C33080B22083884268
:109770000CD949424018208328884449401C80B2B3
:109780000B312880884201D3002028802D887D203D
:10979000C000218B68434018A06302903C480678C3
:1097A00028460A3800B2A673E084002803DA7D2137
:1097B000C9004018E084388830214843FBF743FF54
:1097C00007462620205EFBF733FF3946FBF760FD96
:1097D0007F21C905FBF703FDFBF75EFF81B22C4833
:1097E000761E0180B14201E033E030E001D101207A
:1097F000E072A5841420205EFBF72CFF0746019140
:109800000398FBF73BFF234A234BFBF731FE05464A
:109810000E460298FBF71EFF2A463346FBF71AFE58
:109820003A46019BFBF772FDFBF74AFFE06368468F
:109830000088A0830E480E495030807C6071420041
:10984000633108465130FBF799FC0320207005B0C6
:10985000F0BDFFF73BFA0000E4000020EE0000201E
:109860005800002000040050D9000020DA00002039
:10987000C4110020500D00200000002000D027243B
:10988000F40000200801002070140020E70300000D
:10989000EA000020F853E3A59B843E4070B586B0F3
:1098A00014216846FBF783FC01250F4EED030022CF
:1098B00029463046FDF71BFA01200024019002944E
:1098C0006946009503943046FDF70EF90320019098
:1098D00002946946009503943046FDF705F902208D
:1098E00001F05EF806B070BD000400507047000043
:1098F000F8B5044600206A461080194D55222A709A
:10990000AA226A700322AA70661DEE702A7169711C
:10991000144A49008918AC712246E81DFBF72EFC59
:10992000002007E029186A468978128889186A4653
:109930001180401CB042F5DB611DA81CFCF79EF8AD
:1099400001466846018029190078C8716846407848
:10995000087221460931024800F0EEFAF8BD000015
:10996000B0130020500D002010B51B4CE28A208A55
:109970006178824201D3101AE082E28A608B13463A
:1099800043435B182383132A02D15043401820839A
:10999000208B302148436421643048430F49E06202
:1099A0000968401A0E494018A062FBF753FE0D4AA1
:1099B0000D4BFBF7C5FDFBF783FE0C496062884247
:1099C00002DD4A4280186062002801DA40186062B5
:1099D00007490968486110BDD400002094000020A8
:1099E000F0D8FFFFF853E3A59B843E40FF7F0000C3
:1099F00070140020034A1168382389B29943014347
:109A0000116070470030014010B5FDF77DF910BDC1
:109A100010B59AB034216846FBF7C9FB14210DA894
:109A2000FBF7C5FB1C2112A8FBF7C1FB1B48016813
:109A30000324E402A143C21489180160FDF7C8FBA6
:109A400017480169A143016106200090FF20013001
:109A500002900120039010200490022009904004FD
:109A60000B90000100240C900A946846FDF7A6FEB6
:109A70000F200D9003200E900F941094012111944B
:109A80000DA8FDF705FD8120129003208004189099
:109A9000149412A8FDF7E6FB1AB010BD0070004048
:109AA0004010024015480068FF2101310843134966
:109AB00008600846C068124908401049C860084656
:109AC0000068104908400D49086008468068400851
:109AD00040008860084600680121890488430749DE
:109AE00008600846C068FD21090488430349C8602E
:109AF0000020086104480549886070470010024052
:109B00000C40FF88F6FFF6FE0050000800ED00E074
:109B100070B501F0C9F9244C244DA06404E0FCF7B1
:109B20000FF801F0C1F9A064A842F8D1207801260D
:109B30000525F6032D07002806D001280CD00228A1
:109B400017D003282CD129E0012231462846FDF701
:109B5000CEF8FFF75FFD06E0012231462846FDF70B
:109B6000C6F8FFF733FB002231462846FDF7BFF861
:109B700016E0607A0122401E607231462846FDF7E9
:109B8000B6F8FCF78FF9002231462846FDF7AFF80A
:109B9000607A002804D10120207001E0FFF7A4F8CA
:109BA00001F068F870BD0000580000203001CADEE6
:109BB000818CC907C90F002908D0016849680122B2
:109BC00052049143826A1143026851600222416A41
:109BD0001140022907D101684968D2039143C26A42
:109BE0001143026851600422416A1140042907D1DF
:109BF0000168496812049143026B11430268516085
:109C00000822416A1140082907D1016849681203F6
:109C10009143426B1143026851601022416A114026
:109C2000102907D10168896812029143826B1143A0
:109C3000026891602022416A1140202907D1016801
:109C4000896812029143C26B1143026891604022FD
:109C5000416A1140402915D1016849689203914336
:109C6000026C11430268516001221205016C91429D
:109C700008D101684968032252059143426C11439F
:109C8000026851608022416A1140802907D1016831
:109C9000496812039143826C114302685160704716
:109CA00038B504460020E067FDF728F8054620682F
:109CB00000680821084008280BD114482B460022D0
:109CC00089040090204600F057FB002801D00320B3
:109CD00038BD206800680421084004280BD10B48D7
:109CE0002B46002209050090204600F045FB002885
:109CF00001D00320ECE720206067A06700BF0021AF
:109D00007020015500BF0020E2E70000FFFFFF01C7
:109D1000F8B5184CC826E078002829D160790028C9
:109D200026D101206071144D686B002700281ED0D9
:109D3000686BC821081A15E01048E168405C616949
:109D400088470F480A21008848430E490880E06888
:109D5000401CE060E068C82800DBE760696BC82051
:109D6000401A761EE168814201D0002EE4DC677162
:109D7000F8BD00003C00002000000240880C0020DC
:109D8000E4000020F000002070B5224CE0780028AC
:109D90003FD1207900283CD1012020711E4EF1696D
:109DA00000250906002933DA2156625791420AD16B
:109DB000F06940062CD5A079002829D0A57120890A
:109DC000401C208124E0A179002903D1A0710A2040
:109DD00000F0EDFD00202056CC2148430F494218E9
:109DE000206912181279B262401C00222061A2562A
:109DF000CC235A43895881420ADC25612078401CD3
:109E0000207020780E2800D12570A078401CA0700A
:109E1000257170BD3C000020003801406001002029
:109E200070B50546AC6A00215A20015352200153F7
:109E30002046FEF768F870BDF8B50546AC6A666F57
:109E4000A76F2068806880210840802807D1212ED4
:109E500005D1002152200153204600F064F820680B
:109E6000806840210840402807D1222F05D10021D9
:109E70005A200153204600F034F8E06F10210843C7
:109E8000E0672046FEF73FF8F8BD70B50546AC6ABE
:109E90002868006820210840002817D100215A2096
:109EA000015320680068FF21013188432168086060
:109EB00020688068400840002168886020688068C9
:109EC00040218843216888602020A0672046FEF753
:109ED0001FFA70BD70B50446A56A2846FEF719FA48
:109EE00070BD01680968FF22213291430268116048
:109EF00001688968490849000268916020218167EA
:109F000000210166704710B50446206800684021B2
:109F10008843216808602020606700206066204632
:109F2000FEF778FA10BD01680968C0229143026803
:109F3000116020214167704770B5164CE278002A05
:109F40000CD12279002A09D10122E2700025C8290A
:109F500003DC0222A256002A01DCE57070BD012359
:109F6000E356CC2253430C4AD1500123E356CC266E
:109F700073439B180A460146181DFBF7FFF86078EB
:109F8000401C607060780E2800D16570A078401E7B
:109F9000A070E2E73C00002060010020F0B587B02F
:109FA0000446102004900025002003900026E74975
:109FB0002068884200D100E000BF2169A068084302
:109FC00061690843E1690843074620680068E04981
:109FD000084038432168086020684068032109036D
:109FE0008843E168084321684860A769D749206829
:109FF000884201D0206A0743206880680B2109024B
:10A00000884338432168886000BFD249206888426D
:10A010001CD1D148C0688007800F002806D00128D5
:10A020000AD0022805D003280CD108E001200490B2
:10A030000BE00220049008E00420049005E00820D2
:10A04000049002E01020049000BF46E0C34920685D
:10A0500088421CD1C048C0680C210840002806D0A6
:10A0600004280AD0082805D00C280CD108E00020CC
:10A0700004900BE00220049008E00420049005E026
:10A080000820049002E01020049000BF25E0AF49B2
:10A09000206888421FD1B048C06803218902084067
:10A0A000002808D001218902401A0AD0401A05D0A0
:10A0B000401A0CD108E0002004900BE0022004902C
:10A0C00008E00420049005E00820049002E010203D
:10A0D000049000BF01E01020049000BF9B4920685D
:10A0E000884256D1049804281AD004DC002807D0EE
:10A0F00002281CD108E0082816D0102817D117E034
:10A10000FDF7D0FA064616E0934840380068102163
:10A1100008400009002801D0914E00E0914E0AE06D
:10A12000FDF7E4FA064606E00126F60303E000BF69
:10A130000120039000BF00BF002E0AD060684100DC
:10A140004018B04203D860680003B04202D2012038
:10A150000390F4E0606802903046FF21013100F086
:10A1600018FA626852080023801859410191009042
:10A17000029AFAF7D3FF054603200002854205D371
:10A180007948854202D82068C560D8E00120039054
:10A19000D5E00121C903E06988426FD10498042801
:10A1A0003CD006DC002809D0012813D002284AD16F
:10A1B0001CE008283ED0102845D145E0FDF772FA92
:10A1C000400061684908401802906168FAF790FF02
:10A1D00085B23CE0FDF778FA400061684908401814
:10A1E00002906168FAF784FF85B230E05A4840383F
:10A1F0000068102108400009002807D061684A085B
:10A200005A4BD018FAF774FF85B206E061684A0825
:10A21000574BD018FAF76CFF85B218E0FDF766FAD5
:10A22000400061684908401802906168FAF760FFD1
:10A2300085B20CE061684A0801231B04D018FAF7C4
:10A2400057FF85B203E000BF0120039000BF00BFAD
:10A25000102D0FD3474885420CD846480F38284068
:10A2600005902807400F0599084305900598216837
:10A27000C86064E00120039061E0FFE704980428CF
:10A280003AD006DC002809D0012812D0022847D194
:10A290001AE008283BD0102842D142E0FDF702FA2C
:10A2A00061684908401802906168FAF721FF85B299
:10A2B0003AE0FDF709FA61684908401802906168C0
:10A2C000FAF716FF85B22FE02348403800681021C6
:10A2D00008400009002807D061684A08204BD018C0
:10A2E000FAF706FF85B206E061684A081D4BD018F0
:10A2F000FAF7FEFE85B217E0FDF7F8F96168490844
:10A30000401802906168FAF7F3FE85B20CE06168CC
:10A310004A080123DB03D018FAF7EAFE85B203E00E
:10A3200000BF0120039000BF00BF102D05D31148CE
:10A33000854202D82068C56001E00120039000201A
:10A3400020666066039807B0F0BD0000004800403A
:10A35000F369FFEF00380140401002400044004024
:10A3600000093D000024F400FFFF0F0000127A00F6
:10A370000048E801FFFF0000FFB581B004460D462C
:10A3800017460A9E22E0701C00281FD0FCF7B6FC7E
:10A390000499401AB04201D8002E17D120680068F5
:10A3A000FF21A13188432168086020688068400847
:10A3B00040002168886020206067A06700BF0021FE
:10A3C0007020015500BF032005B0F0BD2068C069B2
:10A3D0002840A84201D1012000E00020B842D2D09C
:10A3E0000020F1E710B5044910200968086202480E
:10A3F000FDF78AFD10BD0000F814002001490D2072
:10A40000887070473C00002010B507480A22018A76
:10A4100051438183FEF712FBFEF7F4FBC822034988
:10A420000348FDF701FF10BDD4000020880C002078
:10A43000F8140020F8B53E4C002321783D4A1D4613
:10A44000082910D0072947D0062950D0052952D015
:10A45000042953D0032954D0002956D0012958D0BB
:10A4600002295AD05BE0A17800264A1F04E0314F50
:10A47000BF5DFB189BB2761C9642F8DB66792779A4
:10A480009A195118E3786278C9188918C9194018BF
:10A49000C0430006000E1AD1012E14D0022E16D190
:10A4A00025482449C018FAF769FE00F0F1FF64203E
:10A4B00000F076FABFF34F8F21492048C860BFF300
:10A4C0004F8F00BFFDE759081046FFF711FA2570BE
:10A4D000E570A570A571F8BDA1795054491CC8B2AA
:10A4E000A071A178491F8842F5D1082001E0607071
:10A4F00007202070F8BDE0700620FAE760710520A3
:10A50000F7E7A070E5700420F3E7552807D1012094
:10A51000EFE7AA2803D10220EBE7032803D0257038
:10A52000E570A570F8BD032020702071F8BD000013
:10A53000CB0000204C130020500D00200400FA0531
:10A5400000ED00E00FB410B503A9044B044A0298D3
:10A5500000F01AF910BC08BC04B01847DDB10008BF
:10A56000200100202021020C01D010211046020AF7
:10A5700001D010460839020901D01046091F82088F
:10A5800001D01046891E420801D0881E7047081A63
:10A590007047F8B582B28BB2040C0D0C10465843CC
:10A5A000002126465E43370C360480197941164651
:10A5B0006E43370C36048019794126466E4389195B
:10A5C000F8BD30B47446641E2578641CAB4200D2DA
:10A5D0001D46635D5B00E31830BC184702E008C805
:10A5E000121F08C1002AFAD170477047002001E00D
:10A5F00001C1121F002AFBD1704708B5002168462F
:10A6000001706B46012202212C2000F087FD0221FF
:10A61000684601706B4601222C2000F07FFD08BDCA
:10A6200038B504466D20694608706B46012207491B
:10A630002E2000F073FD0649002C01D0054A00E0F1
:10A64000054A2E2000F050FD38BD0000060800002D
:10A6500006180000070600000716000038B504467B
:10A660006B4602220021362000F024FCB321230097
:10A67000FFF7A7FF0E0F08153A3A3A3A1C273A3A65
:10A680002F34483A0021684601704078410849005B
:10A6900014E06946087880088000401C04E06946A0
:10A6A000087880088000801C08701DE068460278E9
:10A6B0000A40483202704178802001436846417068
:10A6C00012E0684602780A40027040784106490E5E
:10A6D000F4E7694648780221084303E06946487870
:10A6E000FD210840694648706B4601220021362052
:10A6F00000F014FD012200AB11463620013300F0BA
:10A700000DFD38BD69460878CF21084069462030E4
:10A71000CAE708B5032168464170012101706B4604
:10A7200002220021362000F0F9FC0122D20306218A
:10A730002D2000F0D9FC012000F032F90120FFF7B4
:10A740008DFF08BD08B5020A69464A7008706B465D
:10A75000022204212D2000F0E1FC0320694608704C
:10A760006B46012206212D2000F0D8FC002069460E
:10A7700008706B46012206212D2000F0CFFC0A2133
:10A780002D2000F07DFB08BDFFB58DB004460025EF
:10A7900006E025280AD0109A0F999047641C6D1C7A
:10A7A00020780028F5D1284611B0F0BD00270121FE
:10A7B000484A009700E00743641C23780846203B82
:10A7C00098401042F7D120782E2817D10420074353
:10A7D0006078641C2A280CD10E98641C02C8009171
:10A7E0000E900BE000990A22514330394018641C46
:10A7F00000902078014630390929F3D920780028C3
:10A80000D1D0642808D0692806D075281ED0109AA7
:10A810000F9990476D1C5BE00A200E99019001C9C9
:10A820000E91002802DA40422D2102E0390504D5BC
:10A830002B216A461172012103E0F90704D020217F
:10A84000F7E70BAE0B910DE00021FAE70A200E9915
:10A85000019001C90E91F7E70199FAF749FC3031EF
:10A86000761E31700028F7D103A8801B203001909C
:10A87000780701D5009801E00120009001998842F5
:10A8800001DD401A00E000200027009006E002A849
:10A89000109AC05D0F9990476D1C7F1C0B988742E2
:10A8A000F5DB04E0109A30200F9990476D1C009959
:10A8B000481E00900029F5DC05E03078109A761CDF
:10A8C0000F9990476D1C0199481E01900029F4DCF6
:10A8D000641C65E709280100F8B54A002B4B520DAE
:10A8E000D6182B4A0C460546142E2BDA002E12DA07
:10A8F000284BFAF70BFD00221346FBF731F840D244
:10A90000002C03DA0124E40700253AE0204628431E
:10A9100037D0214C14E0214F0B46F7403B402B43EE
:10A9200031D01C4BFAF7F2FC00221346FBF718F863
:10A9300027D2002C03DD01200005F0400419BC43A0
:10A9400000251EE0332E1EDC33460027143BFF4358
:10A95000DF40384217D00F4BFAF782FD0022134632
:10A96000FAF7FEFF0DD2002C0ADD142E0CD0342095
:10A97000811B012088404019A84200D2641C054672
:10A98000BD4321462846F8BD641CF9E701FCFFFFE2
:10A990009C7500883CE4377E0000F03FFFFF0F000D
:10A9A0007D2110B5C900484300F001F810BD002119
:10A9B00040E000BF00BF00BF00BF00BF00BF00BF3E
:10A9C00000BF00BF00BF00BF00BF00BF00BF00BF8F
:10A9D00000BF00BF00BF00BF00BF00BF00BF00BF7F
:10A9E00000BF00BF00BF00BF00BF00BF00BF00BF6F
:10A9F00000BF00BF00BF00BF00BF00BF00BF00BF5F
:10AA000000BF00BF00BF00BF00BF00BF00BF00BF4E
:10AA100000BF00BF00BF00BF00BF00BF00BF00BF3E
:10AA200000BF00BF00BF00BF00BF00BF00BF00BF2E
:10AA300000BF491C8142BCD370470000FEB50446EC
:10AA40000020019000906079734940000E5A6178AF
:10AA50002578491E7148CFB20163042D77D0072DA8
:10AA600075D000210291217801736C49E3790122AC
:10AA700092058969002B6CD0914381616748217AE6
:10AA80004173217A82698907890B0A438261002117
:10AA9000042000F034FB324661492E2000F024FBF4
:10AAA0003846FFF7BDFD5F4E0522705D81004018FE
:10AAB0005D49431807212B2000F030FB5B490298C9
:10AAC00001220B180B21282000F028FB705D58494B
:10AAD00080000A580C21282000F011FBE07955492C
:10AAE00080004018A1794900425A0221272000F035
:10AAF000FBFA51487E00825B0421272000F0F4FA23
:10AB0000E079002829D0A07804282CD02820694694
:10AB1000087220220621272000F0E6FA02AB01226B
:10AB20002621272000F0FAFA444938014018E1783C
:10AB3000890042580821272000F0E1FAA17A601C20
:10AB4000627A0902114313D016E000E001E001210E
:10AB500088E71143F608816190E7642206212720E7
:10AB600000F0C2FAE0E71020694608720246D1E719
:10AB700033490172090A4172417A007A0A0202439A
:10AB80002021272000F0B0FA2E4F0C2123203A6814
:10AB900000F0B5FAF01982880421232000F0A4FA0D
:10ABA000A07900280BD0E079274901224318002121
:10ABB000212000F0B3FA03200190012000902A0721
:10ABC000120F10010243607800218007000B02433E
:10ABD0000198000502430098400402432079C00612
:10ABE000400902436079C00602431F2000F087FA43
:10ABF000A07861780123084302040848DB0302615E
:10AC0000E179490319430A4302610021082000F059
:10AC100076FA0020FEBD00005CB50008240100208B
:10AC20000428000004B500080C0000202A000020C1
:10AC30000CB500082CB5000838B500083CB5000874
:10AC40004110000024B500082C00002038B50C4647
:10AC500007498A8B002102432C2000F045FA684600
:10AC600004706B46012206212C2000F057FA38BDF3
:10AC70002401002010B5FFF7C0FC10BD10B504463C
:10AC80000421362000F0FCF80121C902002C01D07B
:10AC9000084300E0884302460421362000F02FFAE2
:10ACA00010BD000038B540206946087000210E2014
:10ACB00000F0E6F80446002211460E2000F01FFACC
:10ACC0006B46012200210D2000F028FA074A0021DE
:10ACD0000F2000F014FA00F0EDF9224600210E20BA
:10ACE00000F00DFA02480021017338BDF8FF272457
:10ACF00044010020FEB50546042069460870514C09
:10AD00000020607521462031206348710873A083BC
:10AD10006063A06300F0C8F84B4E206002E000F0D2
:10AD2000C3F82060B042FAD10020FFF797FC00F092
:10AD3000BBF8464E20603078242801D9243806E03C
:10AD40000621FAF7D5F90622101A40010843020637
:10AD500001040A4301020A430243B2607060002109
:10AD60001E2000F0CCF900F09FF820606B46012215
:10AD70000021242000F0D2F91E20FFF7E3FC86B268
:10AD8000300AA0730420FFF7DDFC074600F08CF8C2
:10AD900020603806000E0DD002206946087101AB14
:10ADA000012212212D2000F0B9F9A08B0121090305
:10ADB0000843A08300F078F820600620FFF7C2FC6B
:10ADC00060600720FFF7BEFCA060F006C00E207593
:10ADD00001D110202075C0B200F0DCF9E80707D0DF
:10ADE000FFF797FCA08B0121C9020843A0830AE06A
:10ADF0000521362000F02EF81549084002460521AD
:10AE0000362000F071F90120FFF728FC0021042012
:10AE100000F036F8A0610021262000F031F815215D
:10AE20008903084302460021262000F068F9002229
:10AE30002621362000F058F900F036F82060002076
:10AE4000FEBD0000240100203001CADE0000002009
:10AE5000FFFD000038B5094C89B280B26B46022272
:10AE600000F028F8002806D16846407801026846BC
:10AE70000078081884B2204638BD0000FFFF0000AB
:10AE800038B50024E44389B280B26B46042200F056
:10AE900011F8002806D103216846435C2202D41829
:10AEA000491EFAD5204638BD10B500210846FFF7E7
:10AEB000E7FF10BD38B5002909D0402420436C4677
:10AEC0002070C8B27F2906D8607002200AE0694667
:10AED0000870012006E0802420436C466070C80999
:10AEE000A0700320694600F0ADFA38BD10B51446D5
:10AEF00003460A4621461120FFF7DCFF10BD10B5BE
:10AF00000346052200211520FFF7D4FF10BD10B520
:10AF10000346052200211720FFF7CCFF10BD38B5EE
:10AF2000054600206946087000F0C4F8FF2401348B
:10AF30002246002D01D00322120200210D2000F034
:10AF4000D3F8002D13D06B46012203210F20FFF709
:10AF5000B1FF68460078000709D5FFF7A3FE224637
:10AF600000210D2000F0C0F80020C04338BD0020B3
:10AF700038BD10B5024601210A2000F0C0F810BD0E
:10AF800010B5044600211A20FFF77AFF000D2203B6
:10AF90000005120B024300211A2000F0B0F810BD8A
:10AFA00010B5024602492E2000F09EF810BD0000A8
:10AFB00004180000F8B505466B4601220321042061
:10AFC000FFF778FF0126114C3607002D0DD02A46D9
:10AFD00000210C2000F088F8694608781021084309
:10AFE00069460870A069304307E069460878EF2198
:10AFF000084069460870A069B0430B46A061012271
:10B000000321042000F08AF8F8BD0000240100208C
:10B0100010B502460021182000F066F810BD0000AF
:10B02000F8B50746002568460570B807204C2E463F
:10B0300000280ADA8020694608706B460122002148
:10B040000D2000F06BF801202073F807694608789E
:10B0500021D006210843694608706B460122002171
:10B060000D2000F05BF803210F20FFF7F3FE812194
:10B07000C900084219D04020694608706B46012279
:10B0800000210D2000F04AF80020FFF7F7FD002511
:10B090002673ED4309E002210843694608706B46B8
:10B0A000012200210D2000F039F82846F8BD0000EB
:10B0B000440100201CB56B46012203210F20FFF73D
:10B0C000F9FE684600784022C1091040C9014000DD
:10B0D000814208D0012069460871024601AB032174
:10B0E0000D2000F01BF81CBD08B56B461A70120A43
:10B0F0005A7089B280B2022200F010F808BD38B54B
:10B1000000236C46E254120A5B1C042BFADB89B262
:10B1100080B22346042200F001F838BD38B58024FF
:10B12000002909D0C02528436D462870C8B27F2960
:10B1300007D86870022009E02043694608700120A2
:10B1400004E020436870C809A8700320694600F035
:10B15000B5F938BD10B51446012312189B029A4266
:10B1600002D90020C04310BD0B46821E2146092093
:10B17000FFF7D4FF002010BD10B5054A89051269FC
:10B1800001430A4300210820FFF7B9FF002010BD4A
:10B190002401002038B504466B4601220E212B20E5
:10B1A000FFF788FE68460078E10640094001C90EB5
:10B1B0000143684601706B4601220E212B20FFF7E8
:10B1C000ADFF38BD10B5002142541C06120A2243BF
:10B1D0001B0A491C0429F7DB10BD000013B501232D
:10B1E0001A4669460248FDF795F800981CBD000014
:10B1F000F81400207CB5002425466846FFF77FFE42
:10B2000004206946220E2D02154322020C5C1443D1
:10B21000401EF7D5204629467CBD7CB50024254636
:10B220006846FFF774FE04206946220E2D0215437E
:10B2300022020C5C1443401EF7D5204629467CBDF3
:10B24000FBF76AFDFEF7E4FBFDF70CFC3B493C48CD
:10B25000002522C005608561C5613A490562C1606B
:10B260000838FBF7C1FEFDF7E9FBFDF7CBFCFDF766
:10B27000A7FCFDF7AFFB052601223607D1033046B8
:10B28000FBF735FDFEF730F9FDF77AFAFAF758FCCF
:10B29000FAF726FC0721B015FFF7D8FC2A4C0A2143
:10B2A000208A01224843A083170339463046FBF722
:10B2B0001EFD2348C82225498830FCF7B5FF244EDF
:10B2C0002079002836D0FEF7A3FB2571FAF77CFE23
:10B2D00020700F2809D9012239463046FBF707FDB7
:10B2E000FEF716FC0022394609E0012251033046E0
:10B2F000FBF7FDFCFEF70CFC002201214903304660
:10B30000FBF7F5FCFDF78AF9A08B002801D0401E61
:10B31000A0831048A18B00780843D1D10121C90234
:10B320003046FBF7D7FC0028CAD101210846FBF7BD
:10B3300075FFC5E7FDF772F9C2E70000007C004029
:10B3400070140020FFFF0000D4000020880C0020B3
:10B35000000400504200002010B586B01748FBF7EB
:10B360009EFD14216846F9F722FF1548009003203E
:10B37000019000200290052069460007FBF7B4FB0E
:10B3800069461048FBF7B0FB69460F48FBF7ACFB7A
:10B3900001210846FBF742FFFF2401342046FBF75A
:10B3A0000FFF0A4908680422104308602046FBF793
:10B3B00019FFFBF71FFF06B010BD0000701400203E
:10B3C000FFFF000000040050000800500070004023
:10B3D00010B50122920218491848FAF73DFC1648A8
:10B3E000174902888A4225D001807D21C9008180C9
:10B3F0004910C1800A21018100211E224181D243CE
:10B4000082810122C2810184018241828182C182C2
:10B41000018381831E23C386022303877823438706
:10B420008287C28702464032118451849184C1834D
:10B4300000F02EF810BD0000500D002000FC0008A8
:10B44000AA550000F0B58C460025102605210907F5
:10B450008E620E4C08E067467F5DE760A768FF07D5
:10B46000FCD0E7681F706D1C8542F4DB00200746A6
:10B4700006E0E760A568ED07FCD0E5681D54401CB8
:10B480009042F6D38E610020F0BD000000300140F4
:10B4900070B572B60124074DA40221462846FAF77A
:10B4A000C1FB002804D0224603492846FAF7AAFC2B
:10B4B00062B670BD00FC0008500D0020F0B50025FC
:10B4C000102605279C463F070B46BE620C4C06E043
:10B4D000595DE160A168C907FCD0E1686D1C854237
:10B4E000F6DB002007E06146095CE160A168C9075E
:10B4F000FCD0E168401C9042F5D3BE610020F0BD55
:10B50000003001400000010203040005405C00001F
:10B51000A05C0400C06C0800805C0400E03F1E00DA
:10B52000E07D1E0007A9022570889B880A0016008E
:10B53000010006000100020087008D002D001A3175
:10B5400052001A339A001A351D011A376B003B312D
:10B55000BE003B335E013B3596023B3700009959F4
:10B560009959EB518F421E45142E0080EB51F5285E
:10B570003333E13A703DE13AC235852BC23533337E
:10B58000C235C235AE47E13A5138A33051380000D8
:10B590000000000000000102030406070809000083
:10B5A000000001020304030406080C1018203000F8
:10B5B000D0B500080000002024010000DCA5000830
:10B5C000F4B6000824010020FC180000ECA50008D7
:10B5D0000000000000000000000000000704000957
:10B5E0001E08054008260910400856080540082690
:10B5F0001D040008BE1D040008BED8BC4010080091
:10B60000010000000000C84200000000000000002F
:10B61000000000000000000000000000000000002A
:10B620000000000000000000010000000000000019
:10B630000000000000000000000000005C1200009C
:10B6400000000000000000000000000000000000FA
:10B6500000000000000000000000000000000000EA
:10B6600000000000000000000000000000000000DA
:10B6700000000000000000000000000000000000CA
:10B6800000000000000000000000000000000000BA
:10B69000020204000909010200810000000000000C
:10B6A00001000000000E000000000000000000008B
:10B6B000000000000000000000000000000000008A
:10B6C000000000000000000000000000000000007A
:10B6D000000000000000000000000000000000006A
:10B6E000000000000000000000000000000020003A
:04B6F0000000000056
:04000005080050C1DE
:00000001FF
